:1000000000000814000000000000000000000000D4
:1000100000000000000000000000000000000000E0
:1000200000000000000000000000000000000000D0
:1000300000000000000000000000000000000000C0
:1000400000000000000000000000000000000000B0
:02000004001FDB
:020000040020DA
:10000000A00038D50120B8D20000218A400000B4F9
:1000100003000014FF0365B2BC000094000000144C
:10002000010000B9C0035FD6000040B9C0035FD62D
:10003000E0031EAAC0035FD6FE03002AC0035FD6FA
:10004000C0035FD600000000800A8A5220E4A77235
:10005000F6FFFF171F2003D5FD7BBEA9FD0300910E
:10006000F30B00F9930A8A5233E4A772E003132AD0
:10007000EEFFFF97C0FF073600088A5220E4A77200
:10008000EAFFFF97F30B40F9001C0053FD7BC2A869
:10009000C0035FD61F2003D5FD7BBFA9800A8A520B
:1000A00020E4A772FD030091E0FFFF97000000121B
:1000B000FD7BC1A8C0035FD6FD7BBEA9FD030091F7
:1000C000F35301A9930A8A52F403002A33E4A77276
:1000D000E003132AD5FFFF97C0FF2F36E103142A50
:1000E00000088A52F35341A920E4A772FD7BC2A8FD
:1000F000CCFFFF171F2003D5FD7BBEA9FD03009198
:10010000F30B00F9930A8A5233E4A772E003132A2F
:10011000C6FFFF97C0FF4737F30B40F9FD7BC2A82E
:10012000C0035FD61F2003D5FD7BBEA9FD03009150
:10013000F35301A9F403002A1304805273120051EF
:100140008126D31A210C001220DC001122C00011DC
:100150003F2800714030801AD8FFFF9713FFFF350A
:10016000F35341A900048052FD7BC2A8D3FFFF17BF
:10017000FD7BBFA9FD030091ECFFFF97A00180521A
:10018000CEFFFF97FD7BC1A840018052CBFFFF1738
:10019000FD7BBEA980008A522100805220E4A77214
:1001A000FD030091F30B00F9130080529DFFFF97B0
:1001B00080088A520100805220E4A77299FFFF97BD
:1001C000000C8A520100805220E4A77295FFFF972D
:1001D00080098A526100805220E4A77291FFFF9744
:1001E000000A8A520100805220E4A7728DFFFF9717
:1001F00080088A520100805220E4A77289FFFF978D
:1002000000098A52C118805220E4A77285FFFF9727
:10021000000D8A52C121805220E4A77281FFFF970E
:100220008000805200E4A77280FFFF9702640E12E4
:1002300001008452800080522100A07200E4A77265
:100240004100012A77FFFF978012805201008052FF
:1002500000E4A77273FFFF97E003132A73060011EF
:1002600078FFFF977F5A027181FFFF54001380527D
:100270000100985200E4A7721300805269FFFF97B3
:10028000E003132A730600116EFFFF977F5A027175
:1002900081FFFF54001380520100805200E4A772D6
:1002A00060FFFF97F30B40F9FD7BC2A8000C8A5258
:1002B0006100805220E4A7725AFFFF171F2003D568
:1002C000FD7BBEA9211FA052FD030091F30B00F995
:1002D0001381965213E0A772E003132A51FFFF9790
:1002E000E003132AF30B40F9FD7BC2A801408052C2
:1002F000211FA0724BFFFF170084965200E0A772E7
:100300004AFFFF1700000000FD7BBBA9FD03009121
:10031000F35301A914008052F55B02A91500009067
:10032000F76303A9B5121591F96B04A999FFFF971B
:1003300000CF8A52180080528046A2721700805265
:100340001A008052160080528AFFFF9713008052D5
:1003500038FFFF973901805286FFFF9720098052AE
:1003600056FFFF970009805254FFFF97A008805264
:1003700052FFFF97000B805250FFFF97A001805261
:100380004EFFFF97400180524CFFFF9733FFFF97CE
:100390001FE80071400300541F28007104184D7AB3
:1003A0006003005401781A123F1C017120080054A8
:1003B000610600513F500071A8FEFF54A14A613808
:1003C000620000104188218B20001FD61F2003D51A
:1003D0001FE80071011C00512020801A7F56007117
:1003E000000C00121710172AC00900541BFFFF97BA
:1003F0001FE800717306001101FDFF5433008052A5
:10040000E3FFFF171F2003D55A6F1C5313008052C0
:10041000DFFFFF171F2003D5011C00511FE80071EB
:100420002020801A73060011000C001200101A2AF6
:100430001A3C0012D6FFFF171FE80071011C005183
:100440002020801A000C00121410142A941E00128E
:100450009F060071E0050054940500349F0A007166
:1004600033039F1ACAFFFF17011C00511FE80071D8
:100470002020801A13018052000C00121410142A3C
:10048000941E0012C2FFFF17011C00511FE80071EB
:100490002020801A73060011000C00121610162A74
:1004A000D63E00125603162AB9FFFF171F2003D5A8
:1004B000A001805201FFFF97A0058052FFFEFF9729
:1004C000A0058052FDFEFF97A0018052FBFEFF9722
:1004D00040018052F9FEFF9740018052F7FEFF97DE
:1004E00000009052D5FEFF9700008052F35341A9BF
:1004F000F55B42A9F76343A9F96B44A9FD7BC5A845
:10050000C0035FD61F2003D5D3018052A0FFFF1781
:10051000E003182A1300805216FFFF979CFFFF1775
:10052000F70AC05AE003162AE103172AD802180B6B
:10053000D3018052F802180BD6120011B9FEFF97B2
:0405400093FFFF170F
:1005440008082F2F2F2F271B131313130F0101013B
:0505540001010101019D
:00000001FF
